:100000001CC034C033C09FC131C030C02FC02EC00F
:100010002DC02CC02BC02AC029C035C127C026C086
:1000200025C024C023C03CC03DC029C02AC02BC06D
:100030002CC02DC02EC02FC030C011241FBECFED4C
:10004000CDBF10E0A0E6B0E0E6EAF4E002C0059023
:100050000D92A036B107D9F710E0A0E6B0E001C0DC
:100060001D92AA36B107E1F701D21BC2C9CFE82F12
:10007000F0E0EA30F10598F4ED5EFF4F09948EEC64
:1000800008958EE508958DE108958BE508958BED33
:10009000089586E108958FED08958FE508950895F8
:1000A00087ED089584E1089580991DC081EE94E064
:1000B0000197F1F700C00000809915C080916000A1
:1000C000882329F481E080936000919A03C0109204
:1000D000600091988FE39DE0A3E081509040A040A4
:1000E000E1F700C00000809BFECF81E0C99980E06D
:1000F000882309F465C081E090916000911180E04F
:10010000882309F45DC0A1EEB4E01197F1F700C0B7
:10011000000081E0C99980E0882309F451C081E0A2
:1001200090916000911180E0882309F449C080918A
:100130006600909167000196909367008093660037
:100140008A30910569F410926700109266008091E0
:10015000640090916500019690936500809364001F
:1001600080916400909165008A30910569F4109245
:100170006500109264008091620090916300019686
:10018000909363008093620080916200909163007D
:100190008A30910561F4109265001092640010920B
:1001A00063001092620010926700109266008FE365
:1001B0009DE0A3E081509040A040E1F700C0000026
:1001C000829960C0A1EEB4E01197F1F700C0000081
:1001D00081E0829980E0882309F454C081E0909105
:1001E0006000911180E0882309F44CC08091660082
:1001F0009091670001979093670080936600992320
:100200007CF489E090E09093670080936600809191
:10021000640090916500019790936500809364005D
:10022000809164009091650099237CF489E090E0CE
:1002300090936500809364008091620090916300C8
:100240000197909363008093620080916200909187
:100250006300992374F489E090E0909365008093A3
:100260006400909363008093620090936700809392
:1002700066008FE39DE0A3E081509040A040E1F74D
:1002800000C0000008951F920F920FB60F92112424
:100290002F933F934F935F936F937F938F939F938E
:1002A000AF93BF93EF93FF93809161008F5F809333
:1002B0006100873021F481E08093610010C08330B9
:1002C00021F1843028F4813051F0823059F51BC07F
:1002D000853011F18530F0F0863021F522C09498F8
:1002E0008091680088BB80916600C1DE80936800C1
:1002F00080916400BCDE8093690080916200B7DE6B
:1003000080936A000FC0949A0DC0969880916900FE
:1003100088BB08C0969A06C0959880916A0088BBF1
:1003200001C0959AFF91EF91BF91AF919F918F91ED
:100330007F916F915F914F913F912F910F900FBEE1
:100340000F901F9018951F920F920FB60F921124C5
:100350002F933F934F935F938F939F93AF93BF934D
:1003600080916000813009F074C0809166009091A6
:1003700067000197909367008093660099237CF44F
:1003800089E090E09093670080936600809164001C
:10039000909165000197909365008093640080912F
:1003A00064009091650099239CF489E090E090931B
:1003B000670080936600909365008093640080914D
:1003C00062009091630001979093630080936200B4
:1003D000809162009091630099237CF489E090E021
:1003E000909367008093660090936500809364000B
:1003F00090936300809362002CC021E0009709F085
:1004000020E081E040916600509167004115510560
:1004100009F080E0282330E081E090E04091640022
:10042000509165004115510511F080E090E0822364
:100430009323009771F0109260009198939A8FE344
:1004400092E4AFE081509040A040E1F700C000008E
:100450009398BF91AF919F918F915F914F913F91F1
:100460002F910F900FBE0F901F9018951ABA8FEF13
:100470008BBB87BB8AE781BB85E082BB82E080BF04
:1004800084E083BF83E686BF8CE18EBD81E19AE77D
:1004900095BD84BD89E089BF789482E681BF04DE82
:0604A000FECFF894FFCF2F
:00000001FF
